:1000000088C0B2C056C3B0C0AFC0B3C0ADC0ACC0F2
:10001000ABC0AAC0A9C0A8C068C1A6C0A5C0814580
:1000200086468B479048944997609B619E62A16386
:10003000A464A765AA66AC67AE68B069B280B481F3
:10004000B682B883BA84BB84BD84FF21000000005F
:100050000000000000000000000023456C98C9FF6C
:10006000040714233764A0FFFFFFFFFFFFFFFFFF1C
:10007000FFFFFF00000000000000000023405F7A47
:10008000B4FFFFFFFFFFFF001400081400080E1468
:100090000004080E14000305080E14000305080AE6
:1000A0000E14000305080A0E1014000305080A0EBA
:1000B0001012140008000E00080E0004080E0003C1
:1000C00005080E000305080A0E0004080E101400AF
:1000D000F3F404080E10121400080A0C0E0F10128C
:1000E0001400080EEE1400020304050004140004BA
:1000F0000E1400040810140004080F111400EEED93
:10010000ECEB140E08040004080E00EBECEDEEF32B
:10011000F41411241FBECFE5D1E0DEBFCDBF20E037
:10012000A0E6B0E001C01D92A738B207E1F7E2E611
:10013000F0E085E5808781E08383148212828683E4
:100140001182ADE6B0E08EEF15968C9315978DEF8A
:1001500017968C938BE0818788E58287612C712CC0
:1001600088248A94C3D0DDC24BCF1BBC19BC18BCF9
:100170000895189525B7277E25BF29B7226029BF86
:1001800021E022BF019728F020E188952150E9F76E
:10019000F9CF089588EE93E0EDCF8CE287B986EC35
:1001A00086B9369A3699FECF8FEF80936000089516
:1001B000369A3699FECF95B18091600089270895CF
:1001C000CF93C72D81E0870D8F73782E662D90E039
:1001D0009AD26FEF8C2F90E0CF9195C2FF920F9340
:1001E0001F93CF93DF93F82E0CE610E0C5E7D0E025
:1001F00081E0F81205C0F8016081CE0184D204C00C
:10020000CE0179D2F8018083015011092196CF37B0
:10021000D10571F7DF91CF911F910F91FF90089554
:10022000CFDF81E0DBCF811101C09FCF815090E013
:10023000FC01E45BFF4FE491EBBDFC01E05AFF4F92
:10024000E491E9BDFC01EC58FF4F849188BD08950D
:100250000F931F93CF93C82F8B01CC2359F085E0C8
:10026000E2DFC80187DF81DFC80184DFC80182DFE8
:10027000C150F3CFCF911F910F910895EF92FF924C
:100280000F931F93CF93C8E0E82EF12C062F10E0B8
:1002900084E1C9DFC7016EDF68DFC8016BDFC150D1
:1002A000B9F7CF911F910F91FF90EF9008951F9391
:1002B000CF93DF938FEA87B986EC86B910926000FE
:1002C00010E1C0E0D0E085E090E054DF71DFC80FBE
:1002D000D11D1150C1F7CE0124E0969587952A953E
:1002E000E1F7DF91CF911F91089518958FE384BBBB
:1002F000B99AB89ABC9A81E08ABD83BF9AB59062D8
:100300009ABD9AB590689ABD9FEF9DBD80BF80E66B
:100310008CBD97B328B3892F90E0809590958B7F03
:10032000822B88BBC298AA9A8BB780628BBF8AB790
:1003300085608ABF85B7806285BF789487E790E043
:10034000DAD1853511F06CDF11C0712C872D90E06A
:10035000D2D1682E8F3F19F080E040DF07C0872D93
:1003600091E0970D792E803488F3F6CF80916B0061
:100370001091650000916600C0916300CC2319F0D4
:1003800000E010E088E18F5F90E040E050E068E836
:1003900070E0882379F09B012F5F3F4FF90131977F
:1003A000E491EE2319F0922F961BF6CF8150AB010A
:1003B000B901EFCF892F612F70E0A92FB0E0E82FAE
:1003C000F0E0002321F09D012E1B3F0B05C09F0193
:1003D00021503109260F371F3197E40FF51FF49094
:1003E0002A583F4FF901F082815049F7910F9093BD
:1003F0006100112371F0002329F0292F30E02150F2
:10040000310902C020E030E0F901EA58FF4F81E0F5
:10041000808387E0890F282F2150E22FE91BF0E02D
:10042000E55FFE4FE491A22FB0E0AA58BF4FEC93D6
:100430002913F2CFE82FF0E0EB58FF4F21E0409175
:1004400076003081431320E0821B282F80938600A2
:10045000862D853F78F5382D333060F48F5F682E18
:10046000891708F0612C809187008F5F8F718093CE
:10047000870020C0109287003730B0F430916800B8
:10048000332311F0CC2331F08F5F682E891790F061
:10049000612C10C06916E1F3662019F08150682EB6
:1004A00009C02150622E06C0C111F2CF80916400B4
:1004B000882371F3812C84DE70DEC62DC53F28F4BD
:1004C000D0E0CA58DF4FC881DC2F10E000E0EE24F6
:1004D000E39480918700803190F15CDE1092870078
:1004E000C3E6D0E0C12CD12C81E08C0DFFEFCF1AF8
:1004F000DF0A98819F3F31F4219688E0C816D10425
:1005000099F718C06DE570E0A3DEF601E359FF4FDF
:10051000608088818E25888383DE6FE070E080E2D2
:1005200097DE88818E2588837BDE34DE80916300B0
:10053000882311F3612CC0917600DC2F8EC0CE3E53
:1005400019F463E481E204C0CD3E21F468E284E161
:1005500095DE83C0CC3E11F469E203C0CB3E19F4B2
:1005600062E581E0F5CFC33F41F484E15CDE8AE0DF
:1005700090E000DE88E057DE3DC0C43F59F584E6D8
:1005800090E0F8DD0ADE14DE90E0292F30E0F9017A
:10059000E25EFF4FE491E81710F49E5FF6CFF90199
:1005A000E15EFF4FF4906DE770E08F2D82958695A8
:1005B00087704EDE8EEE92E0DDDD65E070E081E07A
:1005C00047DE85E694E0D6DD6DE770E08F2D8F7114
:1005D0003FDE0FC0CE3F81F4612CF12CF0926B0016
:1005E0001FDE6AEF70E081E033DEF39498E1F912E8
:1005F000F5CFD0DDCFDD31C0CD3F91F4612C8FEF51
:1006000080936C000DDE85E00EDEC4DDC3DD84E189
:100610000ADE4DDE80936C0003DEBCDDBBDDF9CF6E
:100620008D2F01DE44DE20916C00821738F00F5FC1
:10063000093078F0D33068F0D1500AC090E030E053
:1006400022503109821793071CF4DC1708F4DF5F8E
:1006500000E0A3DD84EF91E08DDD10928700A8DD3E
:10066000803990F41F5F183008F433CFD53120F073
:1006700010E0DAE0CAE02DCFD23040F08D2F869521
:100680008695D695D80FCD2F10E023CF6EDD85B798
:10069000877E806185BFF89485B7846885BF8B7F2E
:1006A00085BF85B7806285BF889585B78F7D85BFFB
:1006B000EACF1124882009F01895F89416B855DD72
:1006C000B998B898BC9894E4B2990FC0839485B750
:1006D000877E806185BF91BD85B7846885BF8B7F2C
:1006E00085BF78948895F894EFCF8FE58DBF81E032
:1006F0008EBF1FBEFBDDE199FECF1FBA8EBBE09A15
:1007000099278DB30895262FE199FECF1CBA1FBA01
:100710008EBB2DBB0FB6F894E29AE19A0FBE0196FC
:060720000895F894FFCFDC
:00000001FF
